:030000000211D218
:03000B000200BE32
:03002B000203E0ED
:03005B0002052477
:0300730002051A69
:1000800002030406080C10182030406080020304AC
:1000900006080C101820304080FF0406080C1018C9
:1000A0002030406080A0C000000001010003020277
:1000B000010505020D0505050D0603050202C2AF87
:1000C000C0D0C0E0205A25302F02E47330601A05FA
:1000D00060C37405952540F2956040EE758A78E519
:1000E000257003758A000203D90203CC306306C26F
:1000F00086C291C29585258AC25AE525F4700221EF
:10010000BF0561306013206A19758B00D0E0D0D034
:10011000C286C291C295D2AF32C286C291C2950246
:1001200001AFD26EC26FE565601CC3E561149565D1
:100130004014C26ED26FC3E561956450030201AFF3
:100140007561000201AF206C14C286C291C2957421
:100150001AD5E0FDD290D292D2960201AFC286C2E9
:1001600091C295E53D20E22520E10D207502D29057
:10017000307502D2960201AF20E005D2920201AFA3
:10018000207502D296307502D2900201AF20E1159F
:1001900020E00D207502D290307502D2960201AF98
:1001A000D2920201AF207502D296307502D29075BC
:1001B0008B00D0E0D0D0C286C291C295D2AF32D0EF
:1001C000E0D0D0D2AF3261CCE525600A207502D2F2
:1001D00086307502D295C29161CCE5256002D2913C
:1001E000207502C295307502C28661CCE525600A91
:1001F000207502D295307502D286207502C28630F3
:100200007502C29561CC207502C290307502C2960B
:10021000E525600A207502D286307502D2952075D8
:1002200002C296307502C290C29161CC207502C2A2
:1002300090307502C296207502C296307502C29047
:10024000740ED5E0FDE525600A207502D286307572
:1002500002D295C29161CC207502C290307502C263
:1002600096E525600A207502D286307502D295C2C5
:1002700092C29161CC207502C290307502C296C2C2
:1002800092740ED5E0FDE525600A207502D2863015
:100290007502D295C29161CCC292E5256002D291DD
:1002A000207502C290307502C296207502C2953048
:1002B0007502C28661CCC292207502C2903075026E
:1002C000C296740ED5E0FDE5256002D2912075023C
:1002D000C295307502C28661CCC292E5256002D219
:1002E00091207502C296307502C290207502C295A7
:1002F000307502C28661CCC292207502C2963075FA
:1003000002C290740ED5E0FDE5256002D291207501
:1003100002C295307502C28661CC207502C2963049
:100320007502C290E525600A207502D295307502EB
:10033000D286C292207502C286307502C29561CC07
:10034000207502C296307502C290C292740ED5E03A
:10035000FDE525600A207502D295307502D286200F
:100360007502C286307502C29561CC207502C296B4
:10037000307502C290E525600A207502D29530756D
:1003800002D286207502C290307502C29620750294
:10039000C286307502C29561CC207502C296307556
:1003A00002C290207502C290307502C296740ED5BA
:1003B000E0FDE525600A207502D295307502D286EF
:1003C000207502C286307502C29561CCE525F4F530
:1003D0008A758B00756000D25AD0E0D0D0D2AF328F
:1003E000C2AFC0D0C0E0D2D3C2CEE528600A741F2D
:1003F000552E60491528813D78007900E5803076DA
:1004000001F430E50278FF53DACF20760343DA2097
:1004100030760343DA10C2D8C269E580307601F441
:1004200030E50279FFC3E89970CE3059037528187A
:10043000741F552E60037528188858D268E5296006
:100440000415298150741F552E600543DA01C2D866
:1004500020680281E2E558F8C268741F552E6036A4
:100460007982B70431C3E894F0400374F0F8E8C42B
:0F047000540F28F87984B703028196C313C3137E
:10047F008721200802C313200A06C3C898F8819663
:10048F0028F8500374FFF8C3E8955F5003E55FF851
:10049F00E52C5406703D882230630AC3E522955C33
:1004AF004003855C227882B60429C3E52295244057
:1004BF001278A096400DE52426F52450097524FFE7
:1004CF000204D5852224852425C3E524955C4003A9
:1004DF00855C2520CF09D0E0D0D0C2D3D2AF32C2B5
:1004EF00CF7801E5286008741F552E70021528C3B8
:1004FF00E55894014005755B00A111E55B046002AE
:10050F00055BD0E0D0D0C2D3D2AF32C2AF53917F10
:10051F00C258D2AF32C2AFC0D0C0E0C0F0D2D3A861
:10052F00FBA9FCC2D8306902A18753DACF2076032A
:10053F0043DA1030760343DA20D269E58030760152
:10054F00F420E502A15B88268927E12753DACF2023
:10055F00760343DA2030760343DA10C2D8C26974C7
:10056F001F552E7002E10D7800E580307601F430D2
:10057F00E502E10D8858E10D53DACF20760343DA17
:10058F002030760343DA10C269205902C14153DA91
:10059F00CF20760343DA1030760343DA20C2D8D265
:1005AF006988538954C3E89551F8E99552F9E4FBEA
:1005BF007AFAC3E894C8E994005008E4D2E4FB7ACD
:1005CF000AC114C3E89468E994015008E4D2E3FB2C
:1005DF007A0FC114C3E894D0E994025008E4D2E230
:1005EF00FB7A1EC114C3E894A0E994055008E4D225
:1005FF00E1FB7A3CC114C3E89498E994085006E4EF
:10060F00D2E0FB7A78C3E89555FCE99556FD30E7C3
:10061F0008ECF42401FCEDF4FD7557007008C3ECF1
:10062F009A500375570188558956A853A954885174
:10063F008952C3E89526F8E99527F9307402C1E08D
:10064F00307302C1E0307202C1D9E9C313F9E81364
:10065F00F8307102C1D9E9C313F9E813F830700209
:10066F00C1D9E9C313FDE813FC205918C3EC941C3E
:10067F00ED9402400302070DED7009C3EC94C850CE
:10068F000302072774002077037896E624FAFEE426
:10069F003400FFC3EC9EFCED9FFD500678007900FF
:1006AF00C1E0C3EC94FFED9400400678FF7900C1E0
:1006BF00E0EC856CF0A4C5F0A2F733F879004003A5
:1006CF000206FC78FF79000206FCE9C313F9E81370
:1006DF00F830740EE9600278FFC3E81338F8E43499
:1006EF0000F9C3E894FFE99400400278FF8858D2DC
:1006FF0068205902E10D741FF4552E4BF52E752805
:10070F0018741F552E700375280A305902E127748B
:10071F001F552E600353DAFE752906741F552E7070
:10072F000375290AD0F0D0E0D0D0C2D3D2AF32793E
:10073F0001E1567903E156790AE156791EE15679BE
:10074F0064E15679C8E1567817E4D5E0FDD8FAD9B7
:10075F00F6227A147B7802077D7A107B8C02077D54
:10076F007A0D7BB402077D7A0B7BC802077DAC251F
:10077F007525017902B275E4C292D5E0FDE52560D9
:10078F0002D291D5E0FDC291D5E0FDD292D5E0FD28
:10079F00E525600A207502D286307502D295E56D87
:1007AF00D5E0FD207502C286307502C2957496D5CC
:1007BF00E0FDD9C1EAF8D5E0FDD8FBDBB1C2928CE0
:1007CF002522C37C007D0075F00005F0EA33FAEBBB
:1007DF0033FB50F6EB13FBEA13FAC3E9FFE8FEE82D
:1007EF009AF8E99BF95004EFF9EEF8B3EC33FCED0E
:1007FF0033FDD5F0DFEDF9ECF822E889F08A20D24D
:10080F00D4F8A9F07B0030F70B7BFFF42401F8E953
:10081F00F43400F9E88520F0A4ADF0F8E98520F074
:10082F00A4AFF0FEED2EF974003FFA7C04C3EA1377
:10083F00FAE913F9E813F8DCF48BF030F70AE8F46F
:10084F002401F8E9F43400F9E889F0C2D4F8A9F0EA
:10085F00227882B604030208ECC3E55894014018CD
:0F086F00E54870377805C37994B702027812C351
:10087E00E53B9400E53C984020E5486009855E5DC7
:10088E007562FF756301852224E4F53FF540F5415D
:10089E00F542F543F5480208EC754801C37994E733
:1008AE009402601BE523F43333F913F8E954010481
:1008BE00F9E854FEC39440F8E99400F90208E8E51B
:1008CE0023F433333333F913F8E954070404F9E806
:1008DE0054F8C39440F8E99400F9883F894022E522
:1008EE0048603BC3E53C13F9E53B13F8C3E53F987D
:1008FE00F8E54099F9500CC3E89480E994FF40164E
:10090E00020928C3E8947FE994005003020928786D
:10091E007F7900020928788079FF8844894522E58D
:10092E00486058E5442541F8E5453542F9854520AE
:10093E00E4300701F43543FA30E709C3EA94F04096
:10094E001502096AC3EA940F500302096A78FF7907
:10095E00FF7A0F02096A780079007AF0C3E52495D0
:10096E005C5006E52460092183E54520E70D2183CF
:10097E00E54530E706884189428A4322E5487003FF
:10098E000209ED789EE6FAC3E54433F8E54533F9FE
:10099E001109E930E70BC3E89480E994FF40132175
:1009AE00C4C3E8947FE99400500221C4787F790093
:1009BE0021C4788079FFE820E715C3E52398F84035
:1009CE0009C3E8940140030209EB78010209EBE840
:1009DE00F424012523F840030209EB78FF88462210
:1009EE00E5487003020A4F789FE6FAA842A9431120
:1009FE0009E930E70CC3E89401E994FF4016020AB6
:100A0E0026C3E894FFE994005003020A2678FF7982
:100A1E0000020A26780179FFE920E715C3E546981A
:100A2E00F84009C3E894014003020A4D7800020A17
:100A3E004DE8F424012546F84003020A4D78FF885C
:100A4E002422020AE77883E6F520120F4B75E89010
:100A5E00E5E820ECEDA8BDA9BE120FE3756855754B
:100A6E006900C3740013FD745513FC74552CFC748B
:100A7E00003DFDECFAEDFBC3E89AE99B4014E568F6
:100A8E002455F568E5693400F569EA2CFAEB3DFB6F
:100A9E0080E5AE68AF69C3E56913F9E56813F8C37D
:100AAE00E913F9E813F8E56828F566E56939F5679D
:100ABE007A03C3E913F9E813F8DAF7AA201A7009D2
:100ACE00756800756900020AE71AEA6008EE28FEEA
:100ADE00EF39FFDAF88E688F692275E890227883F5
:100AEE00E6FFE5E820ECF7A8BDA9BE056AC3E56AF6
:100AFE0094084052756A00E97007E56B601B020BA3
:100B0E001BC3E8956B6010E56B5006600C14020B6E
:100B1E00270460F9020B27E56BF56BC3946DF84063
:100B2E0021755CC0C3E89404F84017755C80C3E877
:100B3E009404F8400D755C40C3E89404F8400375C6
:100B4E005C0075BB0B22C3E56AB4070375BB1022AC
:100B5E0030610278323062027878E52C5406601FDC
:100B6E00E879A187F0A4C5F0A2F733F8C3E8955C45
:100B7E004002A85C882288248825306102885E2283
:100B8E00788FE6FFC3EF94055018C3EF94045020FE
:100B9E00C3EF94035028C3EF94025030C3EF940177
:100BAE0050387533A075340F75353C75360561F6C2
:100BBE007533C075341275354075360661F675336A
:100BCE00707534177535D075360761F675334C75FB
:100BDE00341D7535C475360961F6753328753423A1
:100BEE007535B875360B61F685334F853450753BC8
:100BFE0000753C0822A84FA950020C0EA849A94A1C
:100C0E00759100C3E498F594E499F595759104D225
:100C1E005875C820A8CCA9CD75C824AA39AB3A8876
:100C2E0039893AC3E89AF8E99BF9AA3BAB3CC3EB86
:100C3E0013FDEA13FCC3ED13FDEC13FCC3EA9CFA9F
:100C4E00EB9DFBEA28FAEB39FB8A3B8B3C400122F9
:100C5E00753BFF753CFF223058028165759100C3CC
:0F0C6E00E4954BF594E4954CF595759104D258A7
:100C7D00227892E6FF7E10305B027F053063047FA1
:100C8D00037E00A93CA83B7A04C3E913F9E813F8E5
:100C9D00DAF7C3E89EF8E99400F94009C3E8940235
:100CAD00E9940050047802E4F9E9FBE8FAC3E9138A
:100CBD00FDE813FCC3EF9403602EEF20E00DE82C4C
:100CCD00F8E93DF9ECFAEDFB020CE2E828F8E93918
:100CDD00F97A02E4FBC3EF9403400D8A4D8B4E88E5
:100CED0049894A8C4B8D4C22884D894E8A498B4AB5
:100CFD008C4B8D4C22305802A102759100C3E495A6
:100D0D003BF594E4953CF595759104D25822753ECA
:100D1D0000752000020D2A753E00752040D2AF05EA
:100D2D003E20580122759D00E53CC313C313F808FE
:100D3D006030306A06C313C313F808C3E8940A4041
:100D4D0002780A306D08C3E8940440027804C3E5C4
:100D5D003C9408400D759D02C3E53C94104003750D
:100D6D009D03205803D2AF22790F206D027905D251
:100D7D00AF0000C2AF205A0A7932206D02791030CF
:100D8D006FE03063027978C3E58B9940D5E59BF42C
:100D9D00F45440B52002A12AD8C8D2AF22C25B7844
:100DAD009CE6146007E53E147002D25B30630B05C0
:100DBD0038205810753800020DD1205807158115AF
:100DCD008102172422759100C3E4954DF594E495A5
:100DDD004EF595759104D25822AE25305B4F78A310
:100DED00E6FFBF010BD25C752500C286C291C2958C
:100DFD00916A305C03752500305802A1FFBF020BCC
:100E0D00D25C752500C286C291C29578A2B6010D3D
:100E1D00916A305C03752500305802C11FBF030B6A
:100E2D00D25C752500C286C291C295B1D2305C03E9
:100E3D00752500305802C13A305B04C25C8E252204
:100E4D00C2AFC292206A03020E6F90031A206C1279
:100E5D00306E0F207502C296307502C290740ED599
:100E6D00E0FD207502D290307502D296759F5675B1
:100E7D003D02D2AF22C2AF206A03020EA49002D966
:100E8D00306E17C292207502C296307502C29074F0
:100E9D000ED5E0FD020EA79001DA207502C2953045
:100EAD007502C286305A06E5256002D2912075037F
:100EBD00759F76307503759F36753D03D2AF22C28F
:100ECD00AF207502C290307502C296206A03020EE1
:100EDD00EE900298206C0A306E07C292740ED5E027
:100EED00FD207502D296307502D290207503759F44
:100EFD0036307503759F76753D04D2AF22C2AF2093
:100F0D006A03020F2C900257306E17207502C290A3
:100F1D00307502C296C292740ED5E0FD020F2F906D
:100F2D0001C8C291305A0EE525600A207502D2869D
:100F3D00307502D295759F56753D05D2AF22C2AF61
:100F4D00207502C296307502C290206A03020F7599
:100F5D00900206206C12306E0F207502C290307513
:100F6D0002C296740ED5E0FDD292207503759F7660
:100F7D00307503759F36753D06D2AF22C2AF206A1C
:100F8D0003020FB390036B306E1F207502C29030B9
:100F9D007502C296207502C296307502C290740E0B
:100FAD00D5E0FD020FB69001EC207502C2863075BA
:100FBD0002C295305A0EE525600A207502D2953091
:100FCD007502D286207503759F36307503759F7631
:100FDD00753D01D2AF229001C6C286C291C295C2A3
:100FED0090C292C29622C3E54F9535E55095365085
:100FFD0001227890E6FFC3EF94055018C3EF9404D7
:10100D00501BC3EF9403501EC3EF94025021C3EF46
:10101D0094015024C3E54F943CF802104EC3E54FA4
:10102D009428F802104EC3E54F941AF802104EC3DF
:10103D00E54F9412F802104EC3E54F940AF80210D2
:10104D004EE5509400F9884F895022305803021014
:10105D00582278847603788576047886760A788F98
:0E106D00760378907605789576027892760371
:10107B00789B760D7893760578877603789C760146
:10108B00788876017889760178827604788C760177
:10109B00788D7600788E76B478967625789776D09C
:1010AB0078987678789976C8789A7604789D7600D1
:1010BB00227893E6FF756409756501C3BF02097554
:1010CB006405756501021101C3BF030975640575DC
:1010DB006502021101C3BF0409756405756503023E
:1010EB001101C3BF0506756409756507C3BF060605
:1010FB007564007565007887E6FFC26CC3BF030299
:10110B00D26CC26BC3BF0402D26BC26A7418552D6A
:10111B006002D26AC26E6002D26ED26F6002C26F80
:10112B00C2757888E630E102D275C2767889E630EE
:10113B00E102D276C3EF94026008758E01D26D0284
:10114B001152758E00C26D227880E6149000809348
:10115B00789EF67881E61490008093789FF6120FB4
:10116B00E322789BE61490008D9378A0F6120FE3A0
:10117B00227886E61490009A9378A1F6120FE32258
:10118B00789CE6149000A79378A2F6789CE61490CE
:10119B0000AC9378A3F6120FE322227896E6FA7846
:1011AB0097E6FB3077047A007BFFC3EB9AFCC39482
:1011BB008250027C82756C00056CEC856CF0A4C3CC
:1011CB00E5F0948040F222C2D353D9BF7581C0435E
:1011DB00FF8012073E75EF0243B203E5B3240440D0
:1011EB0002F5B37580BF75A44075F17C75D4DF75BE
:1011FB00909875A56775F26775D50075A60175E2B0
:10120B0041120FE3E4F8F6D8FD115F12175411BC2D
:10121B003153316D317C318B31A531A67898866D88
:10122B00120FE375885075890275C8247591047582
:10123B00D84012075212076112074A1207681207A9
:10124B004A12076F12074A121CCD1207521207528D
:10125B0012074E75A82275B80275E69075F61075D3
:10126B009B80759D0375D10E75BC5875BB0B75BAFC
:10127B001175E88012073ED2AF120A5043DA01C251
:10128B00D8C269120752753001D2597A05E55770E9
:10129B00027A05120742E558C3940240EEE52E543C
:1012AB001F855A59F55AB559E2DAE2C25953DACFCA
:1012BB0020760343DA2030760343DA10C2D8C269B2
:1012CB0012074E1207427802741F552E70027800D7
:1012DB00C3E5589840EDC2AF1207611207611207C0
:1012EB0061D2AF120752754700120742788CE6C3E2
:1012FB00940150030213BDE530C394015003021354
:10130B00BD741F552E6035C3E55894FF500302136F
:10131B00BDC2AF120776D2AF12074EC3E558940188
:10132B0050EFC2AF120761120746120761D2AF121C
:10133B00074EC3E55894FF40E9021D527F05D27753
:10134B0031A612074EC2AFC27731A6C3E558947FC0
:10135B00D2AF4068C2AF120776D2AFDFE1C3E55818
:10136B0094057897F61207521217F0121CD57F0AC4
:10137B00D27731A612074EC2AFC27731A6C3E5585A
:10138B00947FD2AF50E8C2AF120761120746120723
:10139B0061D2AFDFDBE55824057896F612075212BF
:1013AB0017F0121D0412074EC3E55894FF40F602C6
:1013BB001D52C3E5589547400385584712074EC346
:1013CB00E5589401400241F4C2AF1207761207763A
:1013DB00120776D2AF120752753000E4F531F532B1
:1013EB000531E531F470360532789AE678281460C9
:1013FB0012785014600D78A014600878F014600314
:10140B00753200C3E53298401415327899866DC257
:10141B00AF120776D2AF7898866D12074E1207423D
:10142B00E5287008741F552E70024194C3E558943B
:10143B000640AD12074EE5287003021294120FE31B
:10144B00E4F522F523F524F525755CFF7885865F99
:10145B00F53FF540F541F542F543F56AF548F52BB7
:0D146B00F52CF55B120B8E756A0875BB1031
:1014780012073E120AE8E5E820ECFBA8BDA9BEE980
:101488007001F8886B120AEC756A0875BB107895BC
:10149800E630E0030214DB7887E6FE760211BC78BA
:1014A80087EEF6D261C2AF120B5E85225C85225DA3
:1014B800D2AFC261752500756200756301D260D232
:1014C80063753800120F4B120F89120C0A120B8E1B
:1014D80002160A7887E6FE76037893E6FD7605110C
:1014E800BC7887EEF67893EDF6D260D261D26E12B0
:1014F8000F4B120F89120B5E12073E120E4D120788
:101508003E12073E120E82120742120ECC120742FA
:10151800120742120F0A120746120F4B1207421205
:10152800073EC261D262120AE8120AEC120B5E751B
:101538006A0875BB10120F89120C03120C7E120F69
:10154800F31158120E4D120C03120C7E120FF311E8
:1015580058120E82120C03120C7E120FF31158123D
:101568000ECC120C03120C7E120FF31158120F0A34
:10157800120C03120C7E120FF31158120F4B120C9F
:1015880003120C7E120FF3C3E54F9535E5509536DF
:10159800400C1158C3E5589401508B021724115878
:1015A800C2627887E6FE760211BC7887EEF685225D
:1015B8005C855E5D855E25756200756301D2637525
:1015C8003800C2AF207502C290307502C2962075ED
:1015D80002C296307502C290742DD5E0FDD2AF12CA
:1015E8000F89120C0A120C65120C7E120D02756A14
:1015F8000075BB0B02160A11BC120F89756A0075BB
:10160800BB0B120D24120DAA120DD2120860120D76
:10161800E6120E4D120C0A120C65120C7E120D0207
:10162800120D1B120DAA120DD21208ED120DE612A0
:101638000E82120C0A120C65120C7E120D02120D8B
:1016480024120DAA120DD212092D120DE6120ECC7B
:10165800120C0A120C65120C7E120D02120D1B12CE
:101668000DAA120DD212098A120DE6120F0A120CD7
:101678000A120C65120C7E120D02120D24120DAA0C
:10168800120DD21209EE120DE6120F4B120C0A12AD
:101698000C65120C7E120D02120D1B120AE8120DB7
:1016A800AA120DD2120AEC120DE6120F89120C0AB8
:1016B800120C65120C7E120D0230632A755CFF75E0
:1016C8005DFF756200756301C3E5389464400AC222
:1016D80063D2647537140216EEC3E55894014003CB
:1016E80002160A021724306419E537147005C2641B
:1016F8000215FFF537C3E5589401400302160A02A4
:101708001724C3E55B94825013741F552E7004E5AB
:10171800286009C3E53C94F05002C10A120FE3782F
:1017280087E6FE760211BC7887EEF6E4F522F5230B
:10173800F524F525F55FC26012073E120FE3741F0A
:10174800552E7006E5287002419461E6901A0D78CE
:1017580020121C00E520B45A0CA3121C00E520B48A
:10176800A503021775115F1217F00217EF7882763A
:1017780004901A077884121C00A308121C00A308FE
:10178800121C00A308121C00A308121C00A30812B4
:101798001C00A308A308A308121C00A308A308A3FD
:1017A80008121C00A308121C00A308A308121C009E
:1017B800A308121C00A308A308121C00A308121CEB
:1017C80000A308121C00A308121C00A308121C0086
:1017D800A308121C00A308121C00A308121C00A3D3
:1017E80008121C00901A2122C2AF121C3F121C19A9
:1017F800901A00740A121C05A37404121C05A37421
:1018080010121C05901A077884121C04A308121CD5
:1018180004A308121C04A308121C04A308121C0425
:10182800A308121C04A308A308A308121C04A308F5
:10183800A308A308121C04A308121C04A308A308E5
:10184800121C04A308121C04A308A308121C04A356
:1018580008121C04A308121C04A308121C04A308E1
:0F186800121C04A308121C04A308121C04A308DA
:10187700121C04A308121C04121C52121C30901ACA
:0218870021221C
:101A00000A0410FFFFFFFF03040A0301015AA501A6
:101A1000FFFF0305FF0305FF0225D0FAFA040D01BD
:021A200000FFC5
:101A4000235475726E6967794145323541232020F0
:101A500023424C48454C4923463333302320202031
:101A60002020202020202020202020202020202076
:101C0000E493F622E6438F01538FFD75EF0275B71B
:101C1000A575B7F1F0538FFE22438F02438F0175F4
:101C2000EF0275B7A575B7F1901A0DF0538FFC222E
:101C3000901A0D745A9105901A0E74A59105227A86
:101C40003079D07820901A409100E520F709A3DA86
:101C5000F7227A3079D0901A40E7910509A3DAF992
:101C600022AB6EA86FBB01057984021CCABB0205BA
:101C70007985021CCABB03057995021CCABB040501
:101C80007986021CCABB0505798F021CCABB0605F2
:101C90007990021CCABB07057992021CCABB0805D1
:101CA000799B021CCABB09057993021CCABB0A05B1
:101CB0007987021CCABB0B05799C021CCABB0C05A8
:101CC0007988021CCA7989021CCAE8F7227C0512AD
:101CD0000752DCFB22C2AF12076112076812076FBE
:101CE00012077612074612076112076812076F1271
:101CF000077612074612076112076812076F12076C
:101D000076D2AF22C2AF12077612076F120768129F
:101D1000076112074612077612076F12076812074B
:101D20006112074612077612076F120768120761E1
:101D3000D2AF22AE6EAF6FC2AF120761120761124F
:101D40000761120746DEF2120776120746DFF8D265
:101D5000AF2291D591CD91CD756E01756F017570E2
:101D600000B1337C05AD58120752C3ED955870F59C
:101D7000C3E55894014009C3E55894FF4032A18E51
:101D800091611217F091D5C2AF75EF1291CDDCD5EC
:101D90000570C3E5709403500280C691CD056FE5D0
:101DA0006E149000B193F808C3E56F98500280AEAE
:101DB00091CD91CD056EC3E56E940E5002809C12BC
:0C1DC000105F1217F0C2AF75EF1291CD4A
:00000001FF
